:040000000200613267
:02000B00804330
:030013000539327A
:05001B00C2A4D2B732BF
:0100230032AA
:10005000C0E085318BE531F46004D2A4C2B7D0E0B2
:100060003275B0FF7590FF7580FF75A0FF758160D8
:10007000D2AAD28A758C00758D00438922D2A9D26A
:10008000B9D2BBD28CD28ED2AFE4F539F53AF53B7A
:10009000F53CF524F525F526F527F5327531FFC237
:1000A00001C200C206C202C203C207C204D20531A5
:1000B0005E3172E541F4702075410F75420A754357
:1000C0000275440F7545FF75466475471075481EE7
:1000D000F535F534F5333144754901754A01754BF1
:1000E00001C2A0C2B5C2B61205931204BD51CD2003
:1000F000001E20031B31FA2007287104711E71A90C
:10010000519D911B9123914B910071CD51BE01EDF9
:10011000911B9123914B9100916871CD51BE512556
:1001200001ED915E7104318601ED90000978337C18
:100130000375961AE6F0A308E596540260FADCF41B
:100140007596022290000078417C0875961AE6F0B8
:10015000A308E596540260FADCF47596022290003A
:100160000078417C0875960AE0F6A308DCFA7596DB
:10017000022290000978337C0375960AE0F6A30802
:10018000DCFA75960222E524752400B410030541BB
:1001900022B40103154122B42003054222B4020314
:1001A000154222B44003054322B40403154322B48C
:1001B0008003054422B40803154422E52575250073
:1001C000B41003054522B40103154522B4200305EC
:1001D0004622B40203154622B4400874012547D4D0
:1001E000F54722B4040874992547D4F54722B48012
:1001F00003054822B40802154822200714E52713F6
:10020000B0B4500DD2077524007525007530FF81FC
:10021000B8300710E52713B3B0B45008C207314413
:10022000D20581BD22300228E541700F20060785E6
:100230004532C20280588546328053D549108541E7
:1002400049E532C395454004C2028024053280202E
:1002500030031DE5437007753200C2038030D54A74
:100260000D85434AE5327004C20380221532801E98
:1002700030061B300018E5427005753246800FD5F8
:100280004B0C85424BC3E532954640021532E532B0
:1002900094118532314003D2AB22C2AB22A2B2B359
:1002A000400122E53C453B453A4539600E753C002E
:1002B000753B00753A00D2A1754019C20122A20017
:1002C00092A3A20692A2D54002C2A10022C290D25D
:1002D00091D292D2938590265326F0D290C291E586
:1002E0009054F0C44526F4F526D291C29285902709
:1002F0005327F0D292C293E59054F0C44527F4F509
:1003000027D29322E5307006852624852725E52609
:1003100045276003854830E5306002153022E52529
:1003200030E002C205E525703CE524606B30050431
:100330007408805AB4100674011532805BB420062C
:10034000740205328052B440047403804BB401043B
:1003500074048044B402047405803DB4040474063B
:100360008036E48033E524702FE5253005047408D9
:10037000801CB410047407801FB420047408801813
:10038000B4400474098011B402047480800AB40873
:100390000474408003E4800020050D752400752559
:1003A000006005D2A1754028226021B4400CC2052E
:1003B0007533007534007535002278357C03540F91
:1003C000FFE6C4FE54F04FF6EE18DCF222A20092D3
:1003D00004A2B0B3720082B4B0019200A204B3824E
:1003E000005010200502312AD202C203E532700308
:1003F000854432A204B0005006D203D205C20222C4
:10040000E4C2AAC539D2AA253CD4F53CE53B340068
:10041000D4F53BE53A3400D4F53A22783379367C8A
:10042000038008783A793D7C038000E6700A77FF04
:100430000908DCF71977F022F754F0700974F047D7
:10044000F7DC01220908E6F7DCFA2279097C067854
:100450003612061679497C06783D12061622794036
:100460007C10784112061622C37499953CFAC37425
:1004700099953BFBC37499953AFCEA2401D4FAEBB5
:100480003400D4FBEC3400D4FCEA2535D4FAEB3547
:1004900034D4FBEC3533D4FC60025012EB4C7013B7
:1004A000EA600BC39547500BD206C201EA22D20183
:1004B000C20622C206C2012290053580039004E5DF
:1004C0001206097C50780080051206447800E893F3
:1004D0001205BE08DCF8229005857C0680EB9005AD
:1004E0008C7C0680E420564F4C42413A202020204C
:1004F00020202020202E2E2E2E2E2E2E2E2E2E2E62
:100500002E2E2E2E2E2E2E2E2E2E2E2E2E204349E9
:100510005441433A2020202020202020202E2E2E1F
:100520002E2E2E2E2E2E2E2E2E2E2E2E2E2E2E2EEB
:100530002E2E2E2E2E552E532E442E542E582E4D0A
:100540002E442E4B2E2E2E2E2E2E2E2E2E2E2E2E98
:100550002E2E2E2E2E2E2E2E2E2E2E2E2E202020E5
:10056000202020202020202020202020202E2E2E61
:100570002E2E2E2E2E2E2E2E2E2E2E2E2E2E2E2E9B
:100580002E2E2E2E2E5354415254202053544F5071
:100590002020207F327EFADEFEDFFA74301205CC96
:1005A0007F32DFFE74301205D374381205D3740C19
:1005B0001205D374011205D374061205D322D2A5F5
:1005C000C2A6D38013D2A5C2A6C3800CC2A6C2A560
:1005D000C38005C2A6C2A5D3F580D2A7C2A7400892
:1005E00022C3D2A5D2A6800CD3C2A5D2A68005C3B1
:1005F000C2A5D2A67580FFD2A7E580C2A75004A2EB
:10060000E740F12274011205D374800205D37C0106
:10061000D2D580067C01C2D5800012064412062382
:10062000DCFB22E620D501C4540F240630E4093057
:1006300007042407800274F6242AB2D520D50108C5
:0A064000090205BEE944800205D35B
